:020000000528D1
:10000800090083161030850028309F00831285016F
:10001800142005150000000005110A3033200C28B3
:1000280085160A3038208512013038201F20643C9C
:10003800031814280800033021280339C6000310C8
:10004800C60DC60D46089F001F14000000000000E2
:10005800000000009F149F182F281E080800C300E6
:100068004120C30B34280800C3003F20C30B3928A4
:1000780008000230422814304228C830C20000006C
:10008800000000000000000000000000C20B432830
:100098000800C8000830C7000514662066206620DE
:1000A8000510662005146620C80D03186620051083
:1000B8006620031C6620C70B562805146620051009
:0E00C800662066200830C900C90B68280800B1
:02400E00E400CC
:00000001FF
